:020000040800F2
:10000000FC7F00200103000805080008090800081B
:100010000D0800081108000815080008010800086C
:100020000108000801080008010800081908000874
:100030001D08000801080008210800084D090008F3
:10004000010800080108000801080008010800086C
:10005000010800080108000801080008010800085C
:10006000010800080108000801080008010800084C
:10007000010800080108000801080008010800083C
:10008000010800080108000801080008010800082C
:10009000010800080108000801080008010800081C
:1000A000010800080108000801080008010800080C
:1000B00001080008010800080108000801080008FC
:1000C00001080008010800080108000801080008EC
:1000D00001080008010800080108000801080008DC
:1000E00001080008010800080108000801080008CC
:1000F00001080008010800080108000801080008BC
:1001000001080008010800080108000801080008AB
:10011000010800080108000801080008010800089B
:10012000010800080108000801080008010800088B
:10013000010800080108000801080008010800087B
:10014000010800080108000801080008010800086B
:10015000010800080108000801080008010800085B
:10016000010800080108000801080008010800084B
:10017000010800080108000801080008010800083B
:10018000010800080108000801080008010800082B
:10019000010800080108000801080008010800081B
:1001A000010800080108000801080008010800080B
:1001B00001080008010800080108000801080008FB
:1001C000010800080000000000000000000000001E
:1001D000000000000000000000000000000000001F
:1001E000000000000000000000000000000000000F
:1001F00000000000000000000000000000000000FF
:100200005A30335F494E3030355F585858585F3058
:100210003030302E303030312E30300000000000D1
:100220004A616E2020352032303234000000000058
:1002300031313A35323A323400000000000000001B
:10024000303030303030303030303030000000006E
:10025000000000000000000000000000000000009E
:10026000000000000000000000000000000000008E
:1002700000000000000000000C0000002000000052
:100280005E89031AE50F4B32181FA64AA178DB6876
:1002900090C155815BA15D6A772868725838DD6F1F
:1002A000000000000000000000000000000000004E
:1002B000000000000000000000000000000000003E
:1002C000000000000000000000000000000000002E
:1002D000000000000000000000000000000000001E
:1002E000000000000000000000000000000000000E
:1002F00000000000000000000000000000000000FE
:1003000008B50E4800F030FB002000F0ADFB00F017
:10031000B1FB002000F0B0FB002000F0B5FB00F0C6
:10032000B5FB00F035FA00F0B1FB00F051FA00F037
:10033000ADFB034B984700F0A9FBFCE7A1170008B1
:100340007D07000855555555555555555555555525
:10035000844641EA000313F003036DD1403A41D3D0
:1003600051F8043B40F8043B51F8043B40F8043B8F
:1003700051F8043B40F8043B51F8043B40F8043B7F
:1003800051F8043B40F8043B51F8043B40F8043B6F
:1003900051F8043B40F8043B51F8043B40F8043B5F
:1003A00051F8043B40F8043B51F8043B40F8043B4F
:1003B00051F8043B40F8043B51F8043B40F8043B3F
:1003C00051F8043B40F8043B51F8043B40F8043B2F
:1003D00051F8043B40F8043B51F8043B40F8043B1F
:1003E000403ABDD2303211D351F8043B40F8043BBF
:1003F00051F8043B40F8043B51F8043B40F8043BFF
:1004000051F8043B40F8043B103AEDD20C3205D3CE
:1004100051F8043B40F8043B043AF9D2043208D0C6
:10042000D2071CBF11F8013B00F8013B01D30B8838
:1004300003806046704700BF082A13D38B078DD016
:1004400010F003038AD0C3F10403D21ADB071CBFE8
:1004500011F8013B00F8013B80D331F8023B20F852
:10046000023B7BE7043AD9D3013A11F8013B00F88B
:10047000013BF9D20B7803704B7843708B78837013
:100480006046704753B94AB9002908BF00281CBF0D
:100490004FF0FF314FF0FF3000F06EB9ADF1080CB6
:1004A0006DE904CE00F006F8DDF804E0DDE9022392
:1004B00004B070472DE9F047089D04468C46002B98
:1004C00040F083808A42174647D9B2FA82F242B19D
:1004D000C2F1200024FA00F09140974040EA010C5C
:1004E00094404FEA1748230CBCFBF8F61FFA87FE2E
:1004F00008FB16C143EA014306FB0EF1994209D9F4
:10050000FB1806F1FF3080F01981994240F2168104
:10051000023E3B445B1AA4B2B3FBF8F008FB103375
:1005200044EA034400FB0EFEA64509D93C1900F13C
:10053000FF3380F00581A64540F2028102383C4439
:1005400040EA0640A4EB0E0400261DB1D44000236F
:10055000C5E900433146BDE8F08702B9FFDEB2FAD3
:1005600082F2002A50D1CB1B4FEA174E1FFA87F8B0
:100570000126B3FBFEFC210C0EFB1C3341EA0341B8
:1005800008FB0CF38B4207D979180CF1FF3002D22B
:100590008B4200F2E9808446C91AA3B2B1FBFEF097
:1005A0000EFB101143EA014408FB00F8A04507D9EF
:1005B0003C1900F1FF3302D2A04500F2D980184661
:1005C000A4EB080440EA0C40BFE78B4209D9002D98
:1005D00000F0B1800026C5E9000130463146BDE893
:1005E000F087B3FA83F6002E4AD18B4202D38242BF
:1005F00000F2B880841A61EB030101208C46002DC3
:10060000A8D0C5E9004CA5E7C2F1200320FA03F603
:10061000974001FA02F04FEA174ED9403043030CDD
:10062000B1FBFEF61FFA87F80EFB161143EA0143F1
:1006300006FB08F1994204FA02F409D9FB1806F105
:10064000FF3C80F08D80994240F28A80023E3B441C
:100650005B1A81B2B3FBFEF00EFB103341EA03419B
:1006600000FB08F38B4207D9791800F1FF3C73D2E5
:100670008B4271D902383944CB1A40EA064678E7F2
:10068000C6F1200C03FA06F422FA0CF31C4320FAFC
:100690000CF701FA06F34FEA144E21FA0CF11F434E
:1006A0003B0CB1FBFEF91FFA84F80EFB191143EA6B
:1006B000014109FB08FA8A4502FA06F200FA06F33C
:1006C00008D9611809F1FF3048D28A4546D9A9F105
:1006D00002092144A1EB0A01BFB2B1FBFEF00EFBFF
:1006E000101147EA014700FB08F8B84507D9E71998
:1006F00000F1FF312ED2B8452CD90238274440EA08
:100700000940A7EB0807A0FB02894F45C6464946AA
:100710001AD317D05DB1B3EB0E0267EB010707FAEE
:100720000CFCF2404CEA0202F740C5E90027002623
:100730003146BDE8F0872E4628460BE70646E9E637
:100740001846FDE64345E5D2B8EB020E69EB04011D
:100750000138DFE70846D2E760468DE78146B9E712
:10076000664675E730464AE7ACF1020C394413E7B8
:1007700002383C4424E700BF704700BF08B500F0D2
:100780007BFD00F08DFD002008BD00BF704700BF5D
:100790000A4B0B48834206D00A4A12F8011B03F8A1
:1007A000011B9842F9D1084B084A934204D000211A
:1007B00003F8011B9342FBD1704700BF00000020EB
:1007C0000800002048180008080000204000002011
:1007D00038B5094C094B9C420CD0251FED1A25F069
:1007E000030585F00305ED43254454F8043D98477F
:1007F000AC42FAD138BD00BF5003000850030008D6
:1008000000BFFDE700BFFDE700BFFDE700BFFDE75C
:1008100000BFFDE700BFFDE700BFFDE700BFFDE74C
:1008200000BFFDE7704700BF704700BF164817497B
:100830000368174A23F4406330B403600B68154D16
:10084000154C43F440630B60136823F020031360DE
:100850002B6843F480632B60236823F440332360C8
:10086000D0F8FC3743F44033C0F8FC37D1F8FC37FC
:1008700023F48073C1F8FC37D2F8FC3743F480339B
:1008800030BCC2F8FC3770470C0002400800024040
:1008900004000240000002400C080240030A03F575
:1008A000801380339B0200F00F0031B1596901229F
:1008B00002FA00F00843586170475A69012101FAB1
:1008C00000F022EA00005861704700BF0C4B0D4851
:1008D0000D4910B400226FF07F441A6004600A6072
:1008E0001A685DF8044B42F004021A601A6842F07C
:1008F00002021A601A6842F001021A60704700BFD3
:1009000010E000E014E000E018E000E038B50D4A27
:100910000D4B1868D2E9004519686FF07F43181A2B
:100920005B1A98428BBFD2E9000140EA04030343FB
:10093000294613F15A0041F10001B4220023FFF7C8
:10094000A1FD38BD1800002018E000E0054930B4D2
:10095000D1E9002312F1807443F10005C1E900459B
:1009600030BC7047180000201749184B0A6842F441
:100970007002F0B40A601A68154F164C164E174DE7
:100980001749002042F001021A6038601A6822F00C
:10099000847222F480321A6026601A6822F480225F
:1009A0001A6040F205732860C4F8FC330B680D4AE6
:1009B0000D4843F080530B601368012143F440431A
:1009C0001360F0BC0170704788ED00E00038024011
:1009D0000838024004380240103000240C3802402D
:1009E0004038024000700040200000201A4A13687E
:1009F00043F48033136013689B0382B003D400BFB9
:100A000013689803FBD5154B1549164A1A600B68F5
:100A1000114A43F414430B60136843F0807313606E
:100A20001368990103D400BF13689B01FBD50C4ADE
:100A3000136823F0030343F00203002113600191C4
:100A4000019B082B06D0136803F00C030193019B54
:100A5000082BF8D102B07047003802400438024039
:100A600008380240085A400708B5FFF7BFFF0020CA
:100A700008BD00BF00207047024A136843F0050319
:100A80001360704730380240704700BF704700BFA6
:100A9000014B01221A7070472100002010B500F0B0
:100AA000DDFB00F0CDFA044600F0DEFB044B1A78C3
:100AB00002B11CB900221A7000BFFDE710BD00BFD3
:100AC00021000020F0B4471E002424F00702E34375
:100AD0000A44D2E9242603F00703DB00C3F1200512
:100AE000DA4006FA05F5203B2A4326FA03F30134DF
:100AF0001A43402C07F8012FE7D1F0BC704700BF24
:100B0000704700BF4368C21801338021702B70B555
:100B100011740446436002D90368DB699847A368EF
:100B200004F1900004F180060021DB009DB229430E
:100B300000F8011DD4E902321B0A43EA0263B04205
:100B40004FEA1222C4E90232C5F30221EDD1236833
:100B50002046DB69BDE87040184700BF036870B5E8
:100B60001B690E460446013E9847002121F007020A
:100B7000CB432244D2E9242503F00703DB00C3F171
:100B80002000DA4005FA00F0203B024325FA03F387
:100B900001311A43402906F8012FE7D170BD00BF8B
:100BA0002DE9F04FADF2A45D0346C54914934FF40F
:100BB000207228A81C46FFF7CBFBC6ABC8A904F1DE
:100BC0000F080B931F460DF5667E4FF0000C89460B
:100BD00000240837254608EB0C06382316F801AF29
:100BE000A3F12002C3F120010AFA03F00AFA02F28B
:100BF0002AFA01F1083B0A4313F1080F45EA0205FE
:100C000044EA0004EAD1BE45C7E900450CF1080CEE
:100C1000DED149460DF5A46CD1E91C4EE3004FEA44
:100C2000D44949EA4E39A20943EA5E73D1E9020583
:100C300083EA090342EA8E628E6C0F68D1F8049051
:100C400053404FEADE484FEACE0242EA547248EA85
:100C50004434F71982EA0402CE6C4FEA10284FEAB6
:100C6000500444EAC57448EA056846EB090988EA75
:100C700004084FEAD01A6E082C0A44EA00644AEAD3
:100C8000456A46EAC070DB1982EA9E1288EA0A06C3
:100C900080EA040042EB090208319B1980EAD51072
:100CA00040EB02028C45C1E91E32B5D1149B903352
:100CB0001D4615930FCD18AC0FC40FCD0FC40FCD2B
:100CC0000FC495E80F0084E80F0026AB0293269B23
:100CD0000E93279B0F93229B0793239B0893249BA0
:100CE0000393259B06931A9B0193DDE918541B9BE4
:100CF00009931E9B0C931F9B0D93DDE92001DDE9F9
:100D00001CEC00950A9413E0079C0394089C06943D
:100D1000009CDDF804E001940A9CDDF824C00891F1
:100D200009941946DDE904340790009310460A94AB
:100D3000029A0B9CF2E90278F4E902564FEA903BE2
:100D4000830C029243EA81334BEA814282EA030B2D
:100D50008B0B8A0CCDE91078CDE9125643EA80431B
:100D600042EA803283EA0208119B139A0B947E199F
:100D7000079C4FEAC05A43EB02094AEA512A009AFB
:100D8000039BCF058BEA0A0A47EA502700EA040BC7
:100D90000A9C1AEB060A23EA00034FEA127688EA55
:100DA00007074FEA8278254683EA0B0248EA94084F
:100DB00046EA041B089C069B47EB090701EA040965
:100DC000009C23EA010383EA09096606019B1AEBEA
:100DD00002022C464FEA157A46EAD516009D8EEAA5
:100DE00003038BEA080B03EA05034AEA05182546C4
:100DF0004FEA847A009C4AEA940A0E9C47EB090762
:100E000012EB0409019A099C0EEA020283EA02032A
:100E10000E938CEA0402009B88EA0A0A0CEA040892
:100E20000F9C8BEA060B4FEA456646EAD31647EB62
:100E300004040E9B27462A400C9C1BEB030B8AEAFA
:100E4000060A82EA08084AEB080A14EB09020D9C1C
:100E500047EB0404234619EB0B04049447EB0A0404
:100E6000039F05940E97029E069F0F97C6ACB4424F
:100E7000CDF830E0CDF834C07FF446AFCDE9202383
:100E8000079B2493DDE90489089B0A9C039F009D2E
:100E9000149A2593019B26971C93069F099B2797DD
:100EA000CDE92201CDE91A541D93CDE91889CDE988
:100EB0001EEC159B1AA802F1D00446464F4603E0EB
:100EC00020150008F0E80267D3E9002112EB0608BC
:100ED00041EB0709E3E80289A342F3D1149C802285
:100EE000002104F1100000F0C9FA002363600DF244
:100EF000A45DBDE8F08F00BF9AB32DE9F8434FF031
:100F0000000804460F461646454600F1100901E068
:100F1000AE4224D9D4E90201636810EB08004344CF
:100F200041F10001802BC4E902014544636004D112
:100F300023682046DB6998476368A6EB0508C3F180
:100F40008002904528BF9046B8F1000FE0D009EB31
:100F500003004246791900F025FAAE42DAD8BDE81E
:100F6000F883704710B50446FFF710FC204610BD0B
:100F700000212DE9F041802204468846C0E9021193
:100F80004160103000F07AFA4646474604F190037B
:100F900004F1D000E3E802679842FBD1BDE8F0819C
:100FA000D0B50446FFF7E4FF15A1D1E9000116A36F
:100FB000D3E9002316A7D7E90067C4E92401C4E9EF
:100FC000262315A1D1E9000115A3D3E90023C4E923
:100FD0002867C4E92A0114A7D7E9006714A1D1E959
:100FE0000001C4E92C2314A3D3E90023C4E92E672C
:100FF000C4E93001C4E93223D0BD00BFAFF30080A3
:1010000008C9BCF367E6096A3BA7CA8485AE67BB1B
:101010002BF894FE72F36E3CF1361D5F3AF54FA546
:10102000D182E6AD7F520E511F6C3E2B8C68059B22
:101030006BBD41FBABD9831F79217E1319CDE05BDA
:10104000F0B50024C5B021460026802214A8002750
:10105000CDE91267119400F011FA2146402234A81C
:1010600000F00CFA604B109310A8FFF781FF4EA11F
:10107000D1E900014EA3D3E90023CDE93401CDE944
:1010800036234DA1D1E900014DA3D3E90023CDE9D9
:101090003801CDE93A234CA1D1E900014CA3D3E9B1
:1010A0000023CDE93C01CDE93E234BA1D1E900016C
:1010B0004BA3D3E90023CDE94001CDE942231198A8
:1010C0004A4E254601E0022D21D8DDE912232044B5
:1010D000121943F100038028CDE912231190254411
:1010E00003D110A8FFF75CFD1198C5F10304C0F10E
:1010F00080018C4228BF0C46002CE4D014AB18446D
:1011000022467119FFF724F9022D1198DDD944AB5D
:10111000034401308022702803F8C02C119002D9BA
:1011200010A8FFF73DFD129B34A8002130ADDB0075
:101130009CB2214300F8011DDDE912321B0A43EA8B
:101140000263A8424FEA1222CDE91232C4F302210F
:10115000EDD110A8FFF724FD0DF1FF35002222F09C
:10116000070144A8D343014451E9101403F00703D5
:10117000DB00C3F12000D94004FA00F0203B01431A
:1011800024FA03F301321943402A05F8011FE6D17E
:101190001749684600F0D6F8B0FA80F0400945B02B
:1011A000F0BD00BFAFF3008008C9BCF367E6096A71
:1011B0003BA7CA8485AE67BB2BF894FE72F36E3CE6
:1011C000F1361D5F3AF54FA5D182E6AD7F520E5143
:1011D0001F6C3E2B8C68059B6BBD41FBABD9831FFD
:1011E00079217E1319CDE05BF0170008A4170008E1
:1011F000A817000808B500F027F8BDE8084000F07F
:1012000025B800BF10B50020FFF780FB0C4A13681B
:10121000C01A002809DB0B4C03F57423217803F571
:101220001073136011B1012905D010BD00F00EF844
:101230000123237010BD00F00DF80023237010BDB2
:101240000400002000000020704700BF012105209D
:10125000FFF724BB00210520FFF720BB01214FF43D
:101260000270FFF71BBB00BF00214FF40270FFF7B5
:1012700015BB00BF704700BF08B562B60020FFF77E
:10128000D5FA0548FFF722FB0020FFF7CBFABDE8AF
:1012900008400020FFF7C8BAA0170008FFF7F6BB08
:1012A0002DE9F041FFF7E6FFFFF7A4FFFFF7F0FBA2
:1012B00072B60020FFF72AFB1F4D00F21D23AB6022
:1012C000286062B61D4C1E4E01274FF000080EE04C
:1012D00000231B01F3589847236806EB031155F8C8
:1012E000332088680244591C45F8332021600020CF
:1012F000FFF70CFB2B68C4F80080C31A002BE7DA59
:101300006B683BB100231B01F358984723680133F6
:101310002360ECE7AB68C01A002802DB27600123DA
:10132000D7E7EB6823B902232360FFF7B7FFCCE7C9
:1013300027600123E7E700BF240000203C000020D5
:1013400010180008032A70B412D940EA0105AD074D
:1013500004460B461ED11946204653F8045B54F848
:10136000046BAE4216D1043A032A20461946F2D83D
:10137000561EA2B10139441E01E0C3180CD014F866
:10138000015F11F8012F9542A6EB0403F5D0A81ACE
:1013900070BC7047561EEDE7184670BC704710468B
:1013A000F6E700BF8842F0B40DD98B1883420AD902
:1013B000841832B1224613F8014D02F8014D9942CA
:1013C000F9D1F0BC70470F2A0ED80346541E002AEC
:1013D000F7D001340C44013B11F8012B03F8012F25
:1013E000A142F9D1F0BC704740EA01039B073FD10D
:1013F000A2F1100323F00F0401F1200727441B0979
:1014000001F1100400F1100554F8106C45F8106C4F
:1014100054F80C6C45F80C6C54F8086C45F8086CE2
:1014200054F8046C45F8046C1034BC4205F1100506
:10143000EAD1013312F00C0F01EB031102F00F049B
:1014400000EB031317D0043C24F0030CA5089C44C4
:101450001C1F0E4656F8047B44F8047F6445F9D1FE
:101460006C1C03EB840301EB840102F00302ADE783
:10147000541E0346ADE72246A8E700BFF0B4860736
:1014800046D0541E002A3CD0CAB2034601E0013CBB
:1014900037D303F8012B9D07F9D1032C2AD9CDB2FC
:1014A00045EA05250F2C45EA054534D9A4F110027B
:1014B00022F00F0C03F120071609674403F1100214
:1014C00042E9045542E902551032BA42F8D1721C81
:1014D00014F00C0F03EB021204F00F0613D0331FAD
:1014E00023F003030433134442F8045B9342FBD11B
:1014F00006F003042CB1CAB21C4403F8012B9C4231
:10150000FBD1F0BC704734461346002CF3D1F8E70A
:1015100014460346C1E71A462646E0E700000000ED
:1015200022AE28D7982F8A42CD65EF239144377198
:101530002F3B4DECCFFBC0B5BCDB8981A5DBB5E90A
:1015400038B548F35BC2563919D005B6F111F159D7
:101550009B4F19AFA4823F9218816DDAD55E1CAB08
:10156000420203A398AA07D8BE6F7045015B83129D
:101570008CB2E44EBE853124E2B4FFD5C37D0C5558
:101580006F897BF2745DBE72B196163BFEB1DE8050
:101590003512C725A706DC9B942669CF74F19BC141
:1015A000D24AF19EC1699BE4E3254F388647BEEFDE
:1015B000B5D58C8BC69DC10F659CAC77CCA10C2496
:1015C00075022B596F2CE92D83E4A66EAA84744A08
:1015D000D4FB41BDDCA9B05CB5531183DA88F97640
:1015E000ABDF66EE52513E981032B42D6DC631A875
:1015F0003F21FB98C82703B0E40EEFBEC77F59BF59
:10160000C28FA83DF30BE0C625A70A934791A7D543
:101610006F8203E05163CA06706E0E0A67292914AF
:10162000FC2FD246850AB72726C9265C38211B2EF7
:10163000ED2AC45AFC6D2C4DDFB3959D130D385324
:10164000DE63AF8B54730A65A8B2773CBB0A6A7637
:10165000E6AEED472EC9C2813B358214852C7292CD
:101660006403F14CA1E8BFA2013042BC4B661AA84A
:101670009197F8D0708B4BC230BE5406A3516CC703
:101680001852EFD619E892D110A96555240699D6BB
:101690002A20715785350EF4B8D1BB3270A06A107C
:1016A000C8D0D2B816C1A41953AB4151086C371E2B
:1016B00099EB8EDF4C774827A8489BE1B5BCB03446
:1016C000635AC9C5B30C1C39CB8A41E34AAAD84E28
:1016D00073E363774FCA9C5BA3B8B2D6F36F2E68EF
:1016E000FCB2EF5DEE828F74602F17436F63A578B5
:1016F00072ABF0A11478C884EC39641A0802C78C64
:10170000281E6323FAFFBE90E9BD82DEEB6C50A475
:101710001579C6B2F7A3F9BE2B5372E3F27871C6FE
:101720009C6126EACE3E27CA07C2C021C7B886D12F
:101730001EEBE0CDD67DDAEA78D16EEE7F4F7DF5F7
:10174000BA6F1772AA67F006A698C8A2C57D630A89
:10175000AE0DF9BE04983F111B471C13350B711BCE
:10176000847D0423F577DB289324C7407BABCA3202
:10177000BCBEC9150ABE9E3C4C0D109CC4671D43DF
:10178000B6423ECBBED4C54C2A7E65FC9C297F590F
:10179000ECFAD63AAB6FCB5F1758474A8C19446CBA
:1017A0000100000061626300DDAF35A193617ABA88
:1017B000CC417349AE20413112E6FA4E89A97EA28E
:1017C0000A9EEEE64B55D39A2192992A274FC1A83B
:1017D00036BA3C23A3FEEBBD454D4423643CE80EE2
:1017E0002A9AC94FA54CA49F0000000000000000E9
:1017F000010B0008650F0008A10F0008F90E000892
:10180000050B00085D0B0008C50A0008A10B0008C5
:1018100005120008F51100086842000000000000F1
:101820009D0A0008910A0008A08601001D02000020
:1018300000000000000000000000000000000000A8
:1018400074ECFF7F010000000100000040420F0027
:1018500000A0F0F700A0F0F700A0F0F700A0F0F76C
:1018600000A0F0F700A0F0F700A0F0F700A0F0F75C
:1018700000A0F0F700A0F0F700A0F0F700A0F0F74C
:1018800000A0F0F700A0F0F700A0F0F700A0F0F73C
:00000001FF
